 FileCase

 Timestamp is 5685d156 (Fri Jan 01 04:07:34 2016)

 Preferred load address is 10000000

 Start         Length     Name                   Class
 0001:00000000 000000f8H .idata$5                CODE
 0001:000000f8 00000004H .CRT$XCA                CODE
 0001:000000fc 00000004H .CRT$XCZ                CODE
 0001:00000100 00000004H .CRT$XIA                CODE
 0001:00000104 0000000cH .CRT$XIC                CODE
 0001:00000110 00000004H .CRT$XIZ                CODE
 0001:00000114 00000004H .CRT$XPA                CODE
 0001:00000118 00000004H .CRT$XPZ                CODE
 0001:0000011c 00000004H .CRT$XTA                CODE
 0001:00000120 00000004H .CRT$XTZ                CODE
 0001:00000128 00002170H .rdata                  CODE
 0001:00002298 000000dcH .rdata$r                CODE
 0001:00002380 0000000cH .rdata$sxdata           CODE
 0001:0000238c 00000004H .rtc$IAA                CODE
 0001:00002390 00000004H .rtc$IZZ                CODE
 0001:00002394 00000004H .rtc$TAA                CODE
 0001:00002398 00000004H .rtc$TZZ                CODE
 0001:000023a0 00006b98H .text                   CODE
 0001:00008f38 00000014H .text$yd                CODE
 0001:00008f50 00000224H .xdata$x                CODE
 0001:00009174 00000014H .idata$2                CODE
 0001:00009188 00000014H .idata$3                CODE
 0001:0000919c 000000f8H .idata$4                CODE
 0001:00009294 00000458H .idata$6                CODE
 0001:000096f0 00000091H .edata                  CODE
 0002:00000000 00000b80H .data                   DATA
 0002:00000b80 00001360H .bss                    DATA
 0003:00000000 00000058H .rsrc$01                DATA
 0003:00000060 00000390H .rsrc$02                DATA

  Address         Publics by Value              Rva+Base       Lib:Object

 0000:00000000       __except_list              00000000     <absolute>
 0000:00000003       ___safe_se_handler_count   00000003     <absolute>
 0000:00000000       ___ImageBase               10000000     <linker-defined>
 0001:00000000       __imp__lstrcpynW@12        10001000     kernel32:KERNEL32.dll
 0001:00000004       __imp__lstrlenW@4          10001004     kernel32:KERNEL32.dll
 0001:00000008       __imp__lstrcatW@8          10001008     kernel32:KERNEL32.dll
 0001:0000000c       __imp__lstrcpyW@8          1000100c     kernel32:KERNEL32.dll
 0001:00000010       __imp__MoveFileW@8         10001010     kernel32:KERNEL32.dll
 0001:00000014       __imp__GetLastError@0      10001014     kernel32:KERNEL32.dll
 0001:00000018       __imp__HeapFree@12         10001018     kernel32:KERNEL32.dll
 0001:0000001c       __imp__HeapAlloc@12        1000101c     kernel32:KERNEL32.dll
 0001:00000020       __imp__GetCurrentThreadId@0 10001020     kernel32:KERNEL32.dll
 0001:00000024       __imp__DecodePointer@4     10001024     kernel32:KERNEL32.dll
 0001:00000028       __imp__GetCommandLineA@0   10001028     kernel32:KERNEL32.dll
 0001:0000002c       __imp__EncodePointer@4     1000102c     kernel32:KERNEL32.dll
 0001:00000030       __imp__RaiseException@16   10001030     kernel32:KERNEL32.dll
 0001:00000034       __imp__IsProcessorFeaturePresent@4 10001034     kernel32:KERNEL32.dll
 0001:00000038       __imp__HeapCreate@12       10001038     kernel32:KERNEL32.dll
 0001:0000003c       __imp__HeapDestroy@4       1000103c     kernel32:KERNEL32.dll
 0001:00000040       __imp__GetProcAddress@8    10001040     kernel32:KERNEL32.dll
 0001:00000044       __imp__GetModuleHandleW@4  10001044     kernel32:KERNEL32.dll
 0001:00000048       __imp__ExitProcess@4       10001048     kernel32:KERNEL32.dll
 0001:0000004c       __imp__WriteFile@20        1000104c     kernel32:KERNEL32.dll
 0001:00000050       __imp__GetStdHandle@4      10001050     kernel32:KERNEL32.dll
 0001:00000054       __imp__GetModuleFileNameW@12 10001054     kernel32:KERNEL32.dll
 0001:00000058       __imp__TlsAlloc@0          10001058     kernel32:KERNEL32.dll
 0001:0000005c       __imp__TlsGetValue@4       1000105c     kernel32:KERNEL32.dll
 0001:00000060       __imp__TlsSetValue@8       10001060     kernel32:KERNEL32.dll
 0001:00000064       __imp__TlsFree@4           10001064     kernel32:KERNEL32.dll
 0001:00000068       __imp__InterlockedIncrement@4 10001068     kernel32:KERNEL32.dll
 0001:0000006c       __imp__SetLastError@4      1000106c     kernel32:KERNEL32.dll
 0001:00000070       __imp__InterlockedDecrement@4 10001070     kernel32:KERNEL32.dll
 0001:00000074       __imp__Sleep@4             10001074     kernel32:KERNEL32.dll
 0001:00000078       __imp__SetHandleCount@4    10001078     kernel32:KERNEL32.dll
 0001:0000007c       __imp__InitializeCriticalSectionAndSpinCount@8 1000107c     kernel32:KERNEL32.dll
 0001:00000080       __imp__GetFileType@4       10001080     kernel32:KERNEL32.dll
 0001:00000084       __imp__GetStartupInfoW@4   10001084     kernel32:KERNEL32.dll
 0001:00000088       __imp__DeleteCriticalSection@4 10001088     kernel32:KERNEL32.dll
 0001:0000008c       __imp__GetModuleFileNameA@12 1000108c     kernel32:KERNEL32.dll
 0001:00000090       __imp__FreeEnvironmentStringsW@4 10001090     kernel32:KERNEL32.dll
 0001:00000094       __imp__WideCharToMultiByte@32 10001094     kernel32:KERNEL32.dll
 0001:00000098       __imp__GetEnvironmentStringsW@0 10001098     kernel32:KERNEL32.dll
 0001:0000009c       __imp__QueryPerformanceCounter@4 1000109c     kernel32:KERNEL32.dll
 0001:000000a0       __imp__GetTickCount@0      100010a0     kernel32:KERNEL32.dll
 0001:000000a4       __imp__GetCurrentProcessId@0 100010a4     kernel32:KERNEL32.dll
 0001:000000a8       __imp__GetSystemTimeAsFileTime@4 100010a8     kernel32:KERNEL32.dll
 0001:000000ac       __imp__HeapSize@12         100010ac     kernel32:KERNEL32.dll
 0001:000000b0       __imp__LeaveCriticalSection@4 100010b0     kernel32:KERNEL32.dll
 0001:000000b4       __imp__EnterCriticalSection@4 100010b4     kernel32:KERNEL32.dll
 0001:000000b8       __imp__UnhandledExceptionFilter@4 100010b8     kernel32:KERNEL32.dll
 0001:000000bc       __imp__SetUnhandledExceptionFilter@4 100010bc     kernel32:KERNEL32.dll
 0001:000000c0       __imp__IsDebuggerPresent@0 100010c0     kernel32:KERNEL32.dll
 0001:000000c4       __imp__TerminateProcess@8  100010c4     kernel32:KERNEL32.dll
 0001:000000c8       __imp__GetCurrentProcess@0 100010c8     kernel32:KERNEL32.dll
 0001:000000cc       __imp__LoadLibraryW@4      100010cc     kernel32:KERNEL32.dll
 0001:000000d0       __imp__GetCPInfo@8         100010d0     kernel32:KERNEL32.dll
 0001:000000d4       __imp__GetACP@0            100010d4     kernel32:KERNEL32.dll
 0001:000000d8       __imp__GetOEMCP@0          100010d8     kernel32:KERNEL32.dll
 0001:000000dc       __imp__IsValidCodePage@4   100010dc     kernel32:KERNEL32.dll
 0001:000000e0       __imp__HeapReAlloc@16      100010e0     kernel32:KERNEL32.dll
 0001:000000e4       __imp__RtlUnwind@16        100010e4     kernel32:KERNEL32.dll
 0001:000000e8       __imp__LCMapStringW@24     100010e8     kernel32:KERNEL32.dll
 0001:000000ec       __imp__MultiByteToWideChar@24 100010ec     kernel32:KERNEL32.dll
 0001:000000f0       __imp__GetStringTypeW@16   100010f0     kernel32:KERNEL32.dll
 0001:000000f4       \177KERNEL32_NULL_THUNK_DATA 100010f4     kernel32:KERNEL32.dll
 0001:000000f8       ___xc_a                    100010f8     LIBCMT:crt0init.obj
 0001:000000fc       ___xc_z                    100010fc     LIBCMT:crt0init.obj
 0001:00000100       ___xi_a                    10001100     LIBCMT:crt0init.obj
 0001:00000110       ___xi_z                    10001110     LIBCMT:crt0init.obj
 0001:00000114       ___xp_a                    10001114     LIBCMT:crt0init.obj
 0001:00000118       ___xp_z                    10001118     LIBCMT:crt0init.obj
 0001:0000011c       ___xt_a                    1000111c     LIBCMT:crt0init.obj
 0001:00000120       ___xt_z                    10001120     LIBCMT:crt0init.obj
 0001:00000128       _MainGuid                  10001128     FileCase.obj
 0001:00000138       _MenuGuid                  10001138     FileCase.obj
 0001:00000148       _DialogGuid                10001148     FileCase.obj
 0001:00000158       ??_C@_1DE@BGKMIKPD@?$AAE?$AAu?$AAg?$AAe?$AAn?$AAe?$AA?5?$AAR?$AAo?$AAs?$AAh?$AAa?$AAl?$AA?5?$AA?$CG?$AA?5?$AAF?$AAa?$AAr?$AA?5?$AAG?$AAr?$AAo?$AAu?$AAp?$AA?$AA@ 10001158     FileCase.obj
 0001:00000190       ??_C@_1FG@IEAGHMHI@?$AAF?$AAi?$AAl?$AAe?$AA?5?$AAn?$AAa?$AAm?$AAe?$AAs?$AA?5?$AAc?$AAa?$AAs?$AAe?$AA?5?$AAc?$AAo?$AAn?$AAv?$AAe?$AAr?$AAs?$AAi?$AAo?$AAn?$AA?5?$AAf?$AAo?$AAr?$AA?5?$AAF@ 10001190     FileCase.obj
 0001:000001e8       ??_C@_1BC@DGHEBOMK@?$AAF?$AAi?$AAl?$AAe?$AAC?$AAa?$AAs?$AAe?$AA?$AA@ 100011e8     FileCase.obj
 0001:000001fc       ??_C@_15NKPPEEJO@?$AA?5?$AA_?$AA?$AA@ 100011fc     FileCase.obj
 0001:00000204       ??_C@_1BA@CAKIGJMA@?$AAW?$AAo?$AAr?$AAd?$AAD?$AAi?$AAv?$AA?$AA@ 10001204     FileCase.obj
 0001:00000214       ??_C@_1BG@DFJACJCJ@?$AAP?$AAr?$AAo?$AAc?$AAe?$AAs?$AAs?$AAD?$AAi?$AAr?$AA?$AA@ 10001214     FileCase.obj
 0001:0000022c       ??_C@_1BM@BNELJCPP@?$AAP?$AAr?$AAo?$AAc?$AAe?$AAs?$AAs?$AAS?$AAu?$AAb?$AAD?$AAi?$AAr?$AA?$AA@ 1000122c     FileCase.obj
 0001:00000248       ??_C@_1BM@HMLICANP@?$AAS?$AAk?$AAi?$AAp?$AAM?$AAi?$AAx?$AAe?$AAd?$AAC?$AAa?$AAs?$AAe?$AA?$AA@ 10001248     FileCase.obj
 0001:00000264       ??_C@_1BO@IKHLKIJC@?$AAC?$AAo?$AAn?$AAv?$AAe?$AAr?$AAt?$AAM?$AAo?$AAd?$AAe?$AAE?$AAx?$AAt?$AA?$AA@ 10001264     FileCase.obj
 0001:00000284       ??_C@_1BI@NPBILFDJ@?$AAC?$AAo?$AAn?$AAv?$AAe?$AAr?$AAt?$AAM?$AAo?$AAd?$AAe?$AA?$AA@ 10001284     FileCase.obj
 0001:0000029c       ??_7?$DialogItemBinding@UFarDialogItem@@@@6B@ 1000129c     filecvt.obj
 0001:000002a4       ??_7?$DialogBuilderBase@UFarDialogItem@@@@6B@ 100012a4     filecvt.obj
 0001:000002c8       ??_7PluginEditFieldBinding@@6B@ 100012c8     filecvt.obj
 0001:000002d0       ??_7PluginDialogBuilder@@6B@ 100012d0     filecvt.obj
 0001:000002f4       ??_7PluginCheckBoxBinding@@6B@ 100012f4     filecvt.obj
 0001:000002fc       ??_7PluginRadioButtonBinding@@6B@ 100012fc     filecvt.obj
 0001:00000304       ??_C@_15EFLNJKHH@?$AA?$CF?$AAu?$AA?$AA@ 10001304     filecvt.obj
 0001:0000030c       ??_7PluginIntEditFieldBinding@@6B@ 1000130c     filecvt.obj
 0001:00000314       ??_7PluginUIntEditFieldBinding@@6B@ 10001314     filecvt.obj
 0001:0000031c       ??_C@_11LOCGONAA@?$AA?$AA@ 1000131c     filecvt.obj
 0001:00000320       ??_C@_1CC@CKMDHNMO@?$AAF?$AAi?$AAl?$AAe?$AAC?$AAa?$AAs?$AAe?$AA_?$AAW?$AAo?$AAr?$AAd?$AAD?$AAi?$AAv?$AA?$AA@ 10001320     filecvt.obj
 0001:00000344       ??_C@_1BC@ENICKDH@?$AAC?$AAo?$AAn?$AAt?$AAe?$AAn?$AAt?$AAs?$AA?$AA@ 10001344     filecvt.obj
 0001:00000358       ??_C@_13JOFGPIOO@?$AA?4?$AA?$AA@ 10001358     ProcessName.obj
 0001:00000360       ??_7bad_alloc@std@@6B@     10001360     LIBCMT:new.obj
 0001:00000368       ??_C@_0P@GHFPNOJB@bad?5allocation?$AA@ 10001368     LIBCMT:new.obj
 0001:00000378       __pRawDllMain              10001378     LIBCMT:dllcrt0.obj
 0001:00000378       __pDefaultRawDllMain       10001378     LIBCMT:dllcrt0.obj
 0001:00000380       ??_7exception@std@@6B@     10001380     LIBCMT:stdexcpt.obj
 0001:00000388       ??_C@_0BC@EOODALEL@Unknown?5exception?$AA@ 10001388     LIBCMT:stdexcpt.obj
 0001:000003a0       ??_7type_info@@6B@         100013a0     LIBCMT:typinfo.obj
 0001:000003c4       ??_C@_0P@MIGLKIOC@CorExitProcess?$AA@ 100013c4     LIBCMT:crt0dat.obj
 0001:000003d4       ??_C@_1BI@BGOHAHKC@?$AAm?$AAs?$AAc?$AAo?$AAr?$AAe?$AAe?$AA?4?$AAd?$AAl?$AAl?$AA?$AA@ 100013d4     LIBCMT:crt0dat.obj
 0001:000003ec       ??_C@_1BO@BKOMIGKJ@?$AAr?$AAu?$AAn?$AAt?$AAi?$AAm?$AAe?$AA?5?$AAe?$AAr?$AAr?$AAo?$AAr?$AA?5?$AA?$AA@ 100013ec     LIBCMT:crt0msg.obj
 0001:0000040c       ??_C@_15JNBOKNOG@?$AA?$AN?$AA?6?$AA?$AA@ 1000140c     LIBCMT:crt0msg.obj
 0001:00000414       ??_C@_1BM@JBBEPPHI@?$AAT?$AAL?$AAO?$AAS?$AAS?$AA?5?$AAe?$AAr?$AAr?$AAo?$AAr?$AA?$AN?$AA?6?$AA?$AA@ 10001414     LIBCMT:crt0msg.obj
 0001:00000430       ??_C@_1BK@KMOMNAAI@?$AAS?$AAI?$AAN?$AAG?$AA?5?$AAe?$AAr?$AAr?$AAo?$AAr?$AA?$AN?$AA?6?$AA?$AA@ 10001430     LIBCMT:crt0msg.obj
 0001:0000044c       ??_C@_1BO@BFCDCGC@?$AAD?$AAO?$AAM?$AAA?$AAI?$AAN?$AA?5?$AAe?$AAr?$AAr?$AAo?$AAr?$AA?$AN?$AA?6?$AA?$AA@ 1000144c     LIBCMT:crt0msg.obj
 0001:00000470       ??_C@_1BOO@KGEDBGAJ@?$AAR?$AA6?$AA0?$AA3?$AA3?$AA?$AN?$AA?6?$AA?9?$AA?5?$AAA?$AAt?$AAt?$AAe?$AAm?$AAp?$AAt?$AA?5?$AAt?$AAo?$AA?5?$AAu?$AAs?$AAe?$AA?5?$AAM?$AAS?$AAI?$AAL?$AA?5?$AAc?$AAo?$AAd@ 10001470     LIBCMT:crt0msg.obj
 0001:00000660       ??_C@_1GG@GOPILAJP@?$AAR?$AA6?$AA0?$AA3?$AA2?$AA?$AN?$AA?6?$AA?9?$AA?5?$AAn?$AAo?$AAt?$AA?5?$AAe?$AAn?$AAo?$AAu?$AAg?$AAh?$AA?5?$AAs?$AAp?$AAa?$AAc?$AAe?$AA?5?$AAf?$AAo?$AAr?$AA?5?$AAl?$AAo@ 10001660     LIBCMT:crt0msg.obj
 0001:000006c8       ??_C@_1MG@ENCOOIDF@?$AAR?$AA6?$AA0?$AA3?$AA1?$AA?$AN?$AA?6?$AA?9?$AA?5?$AAA?$AAt?$AAt?$AAe?$AAm?$AAp?$AAt?$AA?5?$AAt?$AAo?$AA?5?$AAi?$AAn?$AAi?$AAt?$AAi?$AAa?$AAl?$AAi?$AAz?$AAe?$AA?5?$AAt@ 100016c8     LIBCMT:crt0msg.obj
 0001:00000790       ??_C@_1DO@BMFCDCD@?$AAR?$AA6?$AA0?$AA3?$AA0?$AA?$AN?$AA?6?$AA?9?$AA?5?$AAC?$AAR?$AAT?$AA?5?$AAn?$AAo?$AAt?$AA?5?$AAi?$AAn?$AAi?$AAt?$AAi?$AAa?$AAl?$AAi?$AAz?$AAe?$AAd?$AA?$AN?$AA?6?$AA?$AA@ 10001790     LIBCMT:crt0msg.obj
 0001:000007d0       ??_C@_1EK@HHFLMAOL@?$AAR?$AA6?$AA0?$AA2?$AA8?$AA?$AN?$AA?6?$AA?9?$AA?5?$AAu?$AAn?$AAa?$AAb?$AAl?$AAe?$AA?5?$AAt?$AAo?$AA?5?$AAi?$AAn?$AAi?$AAt?$AAi?$AAa?$AAl?$AAi?$AAz?$AAe?$AA?5?$AAh?$AAe@ 100017d0     LIBCMT:crt0msg.obj
 0001:00000820       ??_C@_1GK@MFGOKLAG@?$AAR?$AA6?$AA0?$AA2?$AA7?$AA?$AN?$AA?6?$AA?9?$AA?5?$AAn?$AAo?$AAt?$AA?5?$AAe?$AAn?$AAo?$AAu?$AAg?$AAh?$AA?5?$AAs?$AAp?$AAa?$AAc?$AAe?$AA?5?$AAf?$AAo?$AAr?$AA?5?$AAl?$AAo@ 10001820     LIBCMT:crt0msg.obj
 0001:00000890       ??_C@_1GK@MCAAGJMO@?$AAR?$AA6?$AA0?$AA2?$AA6?$AA?$AN?$AA?6?$AA?9?$AA?5?$AAn?$AAo?$AAt?$AA?5?$AAe?$AAn?$AAo?$AAu?$AAg?$AAh?$AA?5?$AAs?$AAp?$AAa?$AAc?$AAe?$AA?5?$AAf?$AAo?$AAr?$AA?5?$AAs?$AAt@ 10001890     LIBCMT:crt0msg.obj
 0001:00000900       ??_C@_1EM@MAADIHMB@?$AAR?$AA6?$AA0?$AA2?$AA5?$AA?$AN?$AA?6?$AA?9?$AA?5?$AAp?$AAu?$AAr?$AAe?$AA?5?$AAv?$AAi?$AAr?$AAt?$AAu?$AAa?$AAl?$AA?5?$AAf?$AAu?$AAn?$AAc?$AAt?$AAi?$AAo?$AAn?$AA?5?$AAc@ 10001900     LIBCMT:crt0msg.obj
 0001:00000950       ??_C@_1GK@FHCKBEFA@?$AAR?$AA6?$AA0?$AA2?$AA4?$AA?$AN?$AA?6?$AA?9?$AA?5?$AAn?$AAo?$AAt?$AA?5?$AAe?$AAn?$AAo?$AAu?$AAg?$AAh?$AA?5?$AAs?$AAp?$AAa?$AAc?$AAe?$AA?5?$AAf?$AAo?$AAr?$AA?5?$AA_?$AAo@ 10001950     LIBCMT:crt0msg.obj
 0001:000009c0       ??_C@_1FC@ECHBIFBC@?$AAR?$AA6?$AA0?$AA1?$AA9?$AA?$AN?$AA?6?$AA?9?$AA?5?$AAu?$AAn?$AAa?$AAb?$AAl?$AAe?$AA?5?$AAt?$AAo?$AA?5?$AAo?$AAp?$AAe?$AAn?$AA?5?$AAc?$AAo?$AAn?$AAs?$AAo?$AAl?$AAe?$AA?5@ 100019c0     LIBCMT:crt0msg.obj
 0001:00000a18       ??_C@_1EC@JIBHAOPH@?$AAR?$AA6?$AA0?$AA1?$AA8?$AA?$AN?$AA?6?$AA?9?$AA?5?$AAu?$AAn?$AAe?$AAx?$AAp?$AAe?$AAc?$AAt?$AAe?$AAd?$AA?5?$AAh?$AAe?$AAa?$AAp?$AA?5?$AAe?$AAr?$AAr?$AAo?$AAr?$AA?$AN?$AA?6@ 10001a18     LIBCMT:crt0msg.obj
 0001:00000a60       ??_C@_1FK@BEOGODMC@?$AAR?$AA6?$AA0?$AA1?$AA7?$AA?$AN?$AA?6?$AA?9?$AA?5?$AAu?$AAn?$AAe?$AAx?$AAp?$AAe?$AAc?$AAt?$AAe?$AAd?$AA?5?$AAm?$AAu?$AAl?$AAt?$AAi?$AAt?$AAh?$AAr?$AAe?$AAa?$AAd?$AA?5@ 10001a60     LIBCMT:crt0msg.obj
 0001:00000ac0       ??_C@_1FI@LOGNIKDM@?$AAR?$AA6?$AA0?$AA1?$AA6?$AA?$AN?$AA?6?$AA?9?$AA?5?$AAn?$AAo?$AAt?$AA?5?$AAe?$AAn?$AAo?$AAu?$AAg?$AAh?$AA?5?$AAs?$AAp?$AAa?$AAc?$AAe?$AA?5?$AAf?$AAo?$AAr?$AA?5?$AAt?$AAh@ 10001ac0     LIBCMT:crt0msg.obj
 0001:00000b18       ??_C@_1EG@BEHAGFJD@?$AAR?$AA6?$AA0?$AA1?$AA0?$AA?$AN?$AA?6?$AA?9?$AA?5?$AAa?$AAb?$AAo?$AAr?$AAt?$AA?$CI?$AA?$CJ?$AA?5?$AAh?$AAa?$AAs?$AA?5?$AAb?$AAe?$AAe?$AAn?$AA?5?$AAc?$AAa?$AAl?$AAl?$AAe?$AAd@ 10001b18     LIBCMT:crt0msg.obj
 0001:00000b60       ??_C@_1FI@HONFMGBI@?$AAR?$AA6?$AA0?$AA0?$AA9?$AA?$AN?$AA?6?$AA?9?$AA?5?$AAn?$AAo?$AAt?$AA?5?$AAe?$AAn?$AAo?$AAu?$AAg?$AAh?$AA?5?$AAs?$AAp?$AAa?$AAc?$AAe?$AA?5?$AAf?$AAo?$AAr?$AA?5?$AAe?$AAn@ 10001b60     LIBCMT:crt0msg.obj
 0001:00000bb8       ??_C@_1FE@LLNEDJMD@?$AAR?$AA6?$AA0?$AA0?$AA8?$AA?$AN?$AA?6?$AA?9?$AA?5?$AAn?$AAo?$AAt?$AA?5?$AAe?$AAn?$AAo?$AAu?$AAg?$AAh?$AA?5?$AAs?$AAp?$AAa?$AAc?$AAe?$AA?5?$AAf?$AAo?$AAr?$AA?5?$AAa?$AAr@ 10001bb8     LIBCMT:crt0msg.obj
 0001:00000c10       ??_C@_1FK@PGACCAFB@?$AAR?$AA6?$AA0?$AA0?$AA2?$AA?$AN?$AA?6?$AA?9?$AA?5?$AAf?$AAl?$AAo?$AAa?$AAt?$AAi?$AAn?$AAg?$AA?5?$AAp?$AAo?$AAi?$AAn?$AAt?$AA?5?$AAs?$AAu?$AAp?$AAp?$AAo?$AAr?$AAt?$AA?5@ 10001c10     LIBCMT:crt0msg.obj
 0001:00000d20       ??_C@_1EK@MBDPDCGA@?$AAM?$AAi?$AAc?$AAr?$AAo?$AAs?$AAo?$AAf?$AAt?$AA?5?$AAV?$AAi?$AAs?$AAu?$AAa?$AAl?$AA?5?$AAC?$AA?$CL?$AA?$CL?$AA?5?$AAR?$AAu?$AAn?$AAt?$AAi?$AAm?$AAe?$AA?5?$AAL?$AAi?$AAb@ 10001d20     LIBCMT:crt0msg.obj
 0001:00000d6c       ??_C@_15IABLJNFO@?$AA?6?$AA?6?$AA?$AA@ 10001d6c     LIBCMT:crt0msg.obj
 0001:00000d74       ??_C@_17LGKOMLJ@?$AA?4?$AA?4?$AA?4?$AA?$AA@ 10001d74     LIBCMT:crt0msg.obj
 0001:00000d7c       ??_C@_1CO@EAEJAADC@?$AA?$DM?$AAp?$AAr?$AAo?$AAg?$AAr?$AAa?$AAm?$AA?5?$AAn?$AAa?$AAm?$AAe?$AA?5?$AAu?$AAn?$AAk?$AAn?$AAo?$AAw?$AAn?$AA?$DO?$AA?$AA@ 10001d7c     LIBCMT:crt0msg.obj
 0001:00000dac       ??_C@_1DE@JNGNBFGO@?$AAR?$AAu?$AAn?$AAt?$AAi?$AAm?$AAe?$AA?5?$AAE?$AAr?$AAr?$AAo?$AAr?$AA?$CB?$AA?6?$AA?6?$AAP?$AAr?$AAo?$AAg?$AAr?$AAa?$AAm?$AA?3?$AA?5?$AA?$AA@ 10001dac     LIBCMT:crt0msg.obj
 0001:00000de0       ??_C@_1BK@DBDEIDLH@?$AAK?$AAE?$AAR?$AAN?$AAE?$AAL?$AA3?$AA2?$AA?4?$AAD?$AAL?$AAL?$AA?$AA@ 10001de0     LIBCMT:tidtable.obj
 0001:00000dfc       ??_C@_07PEJMOBNF@FlsFree?$AA@ 10001dfc     LIBCMT:tidtable.obj
 0001:00000e04       ??_C@_0M@JCPCPOEF@FlsSetValue?$AA@ 10001e04     LIBCMT:tidtable.obj
 0001:00000e10       ??_C@_0M@GDNOONDI@FlsGetValue?$AA@ 10001e10     LIBCMT:tidtable.obj
 0001:00000e1c       ??_C@_08KNHFBNJ@FlsAlloc?$AA@ 10001e1c     LIBCMT:tidtable.obj
 0001:00000e28       __XcptActTab               10001e28     LIBCMT:winxfltr.obj
 0001:00000eb8       __First_FPE_Indx           10001eb8     LIBCMT:winxfltr.obj
 0001:00000ebc       __Num_FPE                  10001ebc     LIBCMT:winxfltr.obj
 0001:00000ec0       __XcptActTabSize           10001ec0     LIBCMT:winxfltr.obj
 0001:00000ec4       __XcptActTabCount          10001ec4     LIBCMT:winxfltr.obj
 0001:00000ec8       ??_C@_0BI@DFKBFLJE@GetProcessWindowStation?$AA@ 10001ec8     LIBCMT:crtmboxw.obj
 0001:00000ee0       ??_C@_0BK@DEKFELLI@GetUserObjectInformationW?$AA@ 10001ee0     LIBCMT:crtmboxw.obj
 0001:00000efc       ??_C@_0BD@HHGDFDBJ@GetLastActivePopup?$AA@ 10001efc     LIBCMT:crtmboxw.obj
 0001:00000f10       ??_C@_0BA@HNOPNCHB@GetActiveWindow?$AA@ 10001f10     LIBCMT:crtmboxw.obj
 0001:00000f20       ??_C@_0M@DLDCCGNP@MessageBoxW?$AA@ 10001f20     LIBCMT:crtmboxw.obj
 0001:00000f2c       ??_C@_1BG@GOEBHBDC@?$AAU?$AAS?$AAE?$AAR?$AA3?$AA2?$AA?4?$AAD?$AAL?$AAL?$AA?$AA@ 10001f2c     LIBCMT:crtmboxw.obj
 0001:00000f44       ??_C@_1BC@GDGBMEMK@?$AAH?$AAH?$AA?3?$AAm?$AAm?$AA?3?$AAs?$AAs?$AA?$AA@ 10001f44     LIBCMT:nlsdata2.obj
 0001:00000f58       ??_C@_1CI@KNAKOEBC@?$AAd?$AAd?$AAd?$AAd?$AA?0?$AA?5?$AAM?$AAM?$AAM?$AAM?$AA?5?$AAd?$AAd?$AA?0?$AA?5?$AAy?$AAy?$AAy?$AAy?$AA?$AA@ 10001f58     LIBCMT:nlsdata2.obj
 0001:00000f80       ??_C@_1BC@IEBCMHCM@?$AAM?$AAM?$AA?1?$AAd?$AAd?$AA?1?$AAy?$AAy?$AA?$AA@ 10001f80     LIBCMT:nlsdata2.obj
 0001:00000f94       ??_C@_15CLMNNGEL@?$AAP?$AAM?$AA?$AA@ 10001f94     LIBCMT:nlsdata2.obj
 0001:00000f9c       ??_C@_15ODEHAHHF@?$AAA?$AAM?$AA?$AA@ 10001f9c     LIBCMT:nlsdata2.obj
 0001:00000fa4       ??_C@_1BC@FEMKIFH@?$AAD?$AAe?$AAc?$AAe?$AAm?$AAb?$AAe?$AAr?$AA?$AA@ 10001fa4     LIBCMT:nlsdata2.obj
 0001:00000fb8       ??_C@_1BC@BGLIFPF@?$AAN?$AAo?$AAv?$AAe?$AAm?$AAb?$AAe?$AAr?$AA?$AA@ 10001fb8     LIBCMT:nlsdata2.obj
 0001:00000fcc       ??_C@_1BA@EPANDLNG@?$AAO?$AAc?$AAt?$AAo?$AAb?$AAe?$AAr?$AA?$AA@ 10001fcc     LIBCMT:nlsdata2.obj
 0001:00000fdc       ??_C@_1BE@DKAAMBJL@?$AAS?$AAe?$AAp?$AAt?$AAe?$AAm?$AAb?$AAe?$AAr?$AA?$AA@ 10001fdc     LIBCMT:nlsdata2.obj
 0001:00000ff0       ??_C@_1O@PAHLKOAC@?$AAA?$AAu?$AAg?$AAu?$AAs?$AAt?$AA?$AA@ 10001ff0     LIBCMT:nlsdata2.obj
 0001:00001000       ??_C@_19BIFMLPCD@?$AAJ?$AAu?$AAl?$AAy?$AA?$AA@ 10002000     LIBCMT:nlsdata2.obj
 0001:0000100c       ??_C@_19EPFLPGAP@?$AAJ?$AAu?$AAn?$AAe?$AA?$AA@ 1000200c     LIBCMT:nlsdata2.obj
 0001:00001018       ??_C@_1M@GJNLMHFD@?$AAA?$AAp?$AAr?$AAi?$AAl?$AA?$AA@ 10002018     LIBCMT:nlsdata2.obj
 0001:00001024       ??_C@_1M@IKEENEDF@?$AAM?$AAa?$AAr?$AAc?$AAh?$AA?$AA@ 10002024     LIBCMT:nlsdata2.obj
 0001:00001030       ??_C@_1BC@JGDDFFAM@?$AAF?$AAe?$AAb?$AAr?$AAu?$AAa?$AAr?$AAy?$AA?$AA@ 10002030     LIBCMT:nlsdata2.obj
 0001:00001044       ??_C@_1BA@EFMEIEBA@?$AAJ?$AAa?$AAn?$AAu?$AAa?$AAr?$AAy?$AA?$AA@ 10002044     LIBCMT:nlsdata2.obj
 0001:00001054       ??_C@_17EGKACKIF@?$AAD?$AAe?$AAc?$AA?$AA@ 10002054     LIBCMT:nlsdata2.obj
 0001:0000105c       ??_C@_17BBDMLCIG@?$AAN?$AAo?$AAv?$AA?$AA@ 1000205c     LIBCMT:nlsdata2.obj
 0001:00001064       ??_C@_17FNLKOI@?$AAO?$AAc?$AAt?$AA?$AA@ 10002064     LIBCMT:nlsdata2.obj
 0001:0000106c       ??_C@_17HCHCOKMG@?$AAS?$AAe?$AAp?$AA?$AA@ 1000206c     LIBCMT:nlsdata2.obj
 0001:00001074       ??_C@_17ICPELBCN@?$AAA?$AAu?$AAg?$AA?$AA@ 10002074     LIBCMT:nlsdata2.obj
 0001:0000107c       ??_C@_17IJPCKHK@?$AAJ?$AAu?$AAl?$AA?$AA@ 1000207c     LIBCMT:nlsdata2.obj
 0001:00001084       ??_C@_17KCJGOCPB@?$AAJ?$AAu?$AAn?$AA?$AA@ 10002084     LIBCMT:nlsdata2.obj
 0001:0000108c       ??_C@_17PNNKMEED@?$AAM?$AAa?$AAy?$AA?$AA@ 1000208c     LIBCMT:nlsdata2.obj
 0001:00001094       ??_C@_17LFPOIHDD@?$AAA?$AAp?$AAr?$AA?$AA@ 10002094     LIBCMT:nlsdata2.obj
 0001:0000109c       ??_C@_17CKNLEDEC@?$AAM?$AAa?$AAr?$AA?$AA@ 1000209c     LIBCMT:nlsdata2.obj
 0001:000010a4       ??_C@_17LMDJEKJN@?$AAF?$AAe?$AAb?$AA?$AA@ 100020a4     LIBCMT:nlsdata2.obj
 0001:000010ac       ??_C@_17DKNBKCHM@?$AAJ?$AAa?$AAn?$AA?$AA@ 100020ac     LIBCMT:nlsdata2.obj
 0001:000010b4       ??_C@_1BC@ENMNNPAJ@?$AAS?$AAa?$AAt?$AAu?$AAr?$AAd?$AAa?$AAy?$AA?$AA@ 100020b4     LIBCMT:nlsdata2.obj
 0001:000010c8       ??_C@_1O@PDICJHAG@?$AAF?$AAr?$AAi?$AAd?$AAa?$AAy?$AA?$AA@ 100020c8     LIBCMT:nlsdata2.obj
 0001:000010d8       ??_C@_1BC@HHMNLIHE@?$AAT?$AAh?$AAu?$AAr?$AAs?$AAd?$AAa?$AAy?$AA?$AA@ 100020d8     LIBCMT:nlsdata2.obj
 0001:000010ec       ??_C@_1BE@EBOGMDOH@?$AAW?$AAe?$AAd?$AAn?$AAe?$AAs?$AAd?$AAa?$AAy?$AA?$AA@ 100020ec     LIBCMT:nlsdata2.obj
 0001:00001100       ??_C@_1BA@ENFBFFEK@?$AAT?$AAu?$AAe?$AAs?$AAd?$AAa?$AAy?$AA?$AA@ 10002100     LIBCMT:nlsdata2.obj
 0001:00001110       ??_C@_1O@MMNBFLIA@?$AAM?$AAo?$AAn?$AAd?$AAa?$AAy?$AA?$AA@ 10002110     LIBCMT:nlsdata2.obj
 0001:00001120       ??_C@_1O@IHNHDHPB@?$AAS?$AAu?$AAn?$AAd?$AAa?$AAy?$AA?$AA@ 10002120     LIBCMT:nlsdata2.obj
 0001:00001130       ??_C@_17GGIBDPIH@?$AAS?$AAa?$AAt?$AA?$AA@ 10002130     LIBCMT:nlsdata2.obj
 0001:00001138       ??_C@_17HFOLPPLP@?$AAF?$AAr?$AAi?$AA?$AA@ 10002138     LIBCMT:nlsdata2.obj
 0001:00001140       ??_C@_17PDPHAADD@?$AAT?$AAh?$AAu?$AA?$AA@ 10002140     LIBCMT:nlsdata2.obj
 0001:00001148       ??_C@_17CJEDCEPE@?$AAW?$AAe?$AAd?$AA?$AA@ 10002148     LIBCMT:nlsdata2.obj
 0001:00001150       ??_C@_17BMKGEGOJ@?$AAT?$AAu?$AAe?$AA?$AA@ 10002150     LIBCMT:nlsdata2.obj
 0001:00001158       ??_C@_17KBOMKBF@?$AAM?$AAo?$AAn?$AA?$AA@ 10002158     LIBCMT:nlsdata2.obj
 0001:00001160       ??_C@_17MBGCMIPB@?$AAS?$AAu?$AAn?$AA?$AA@ 10002160     LIBCMT:nlsdata2.obj
 0001:00001168       ??_C@_08JCCMCCIL@HH?3mm?3ss?$AA@ 10002168     LIBCMT:nlsdata2.obj
 0001:00001174       ??_C@_0BE@CKGJFCPC@dddd?0?5MMMM?5dd?0?5yyyy?$AA@ 10002174     LIBCMT:nlsdata2.obj
 0001:00001188       ??_C@_08BPBNCDIB@MM?1dd?1yy?$AA@ 10002188     LIBCMT:nlsdata2.obj
 0001:00001194       ??_C@_02CJNFDJBF@PM?$AA@   10002194     LIBCMT:nlsdata2.obj
 0001:00001198       ??_C@_02DEDBPAFC@AM?$AA@   10002198     LIBCMT:nlsdata2.obj
 0001:0000119c       ??_C@_08EDHMEBNP@December?$AA@ 1000219c     LIBCMT:nlsdata2.obj
 0001:000011a8       ??_C@_08HCHEGEOA@November?$AA@ 100021a8     LIBCMT:nlsdata2.obj
 0001:000011b4       ??_C@_07JJNFCEND@October?$AA@ 100021b4     LIBCMT:nlsdata2.obj
 0001:000011bc       ??_C@_09BHHEALKD@September?$AA@ 100021bc     LIBCMT:nlsdata2.obj
 0001:000011c8       ??_C@_06LBBHFDDG@August?$AA@ 100021c8     LIBCMT:nlsdata2.obj
 0001:000011d0       ??_C@_04MIEPOIFP@July?$AA@ 100021d0     LIBCMT:nlsdata2.obj
 0001:000011d8       ??_C@_04CNLMGBGM@June?$AA@ 100021d8     LIBCMT:nlsdata2.obj
 0001:000011e0       ??_C@_05DMJDNLEJ@April?$AA@ 100021e0     LIBCMT:nlsdata2.obj
 0001:000011e8       ??_C@_05HPCKOFNC@March?$AA@ 100021e8     LIBCMT:nlsdata2.obj
 0001:000011f0       ??_C@_08GNJGEPFN@February?$AA@ 100021f0     LIBCMT:nlsdata2.obj
 0001:000011fc       ??_C@_07CGJPFGJA@January?$AA@ 100021fc     LIBCMT:nlsdata2.obj
 0001:00001204       ??_C@_03MKABNOCG@Dec?$AA@  10002204     LIBCMT:nlsdata2.obj
 0001:00001208       ??_C@_03JPJOFNIA@Nov?$AA@  10002208     LIBCMT:nlsdata2.obj
 0001:0000120c       ??_C@_03BMAOKBAD@Oct?$AA@  1000220c     LIBCMT:nlsdata2.obj
 0001:00001210       ??_C@_03GGCAPAJC@Sep?$AA@  10002210     LIBCMT:nlsdata2.obj
 0001:00001214       ??_C@_03IFJFEIGA@Aug?$AA@  10002214     LIBCMT:nlsdata2.obj
 0001:00001218       ??_C@_03LBGABGKK@Jul?$AA@  10002218     LIBCMT:nlsdata2.obj
 0001:0000121c       ??_C@_03IDFGHECI@Jun?$AA@  1000221c     LIBCMT:nlsdata2.obj
 0001:00001220       ??_C@_03CNMDKL@May?$AA@    10002220     LIBCMT:nlsdata2.obj
 0001:00001224       ??_C@_03LEOLGMJP@Apr?$AA@  10002224     LIBCMT:nlsdata2.obj
 0001:00001228       ??_C@_03ODNJBKGA@Mar?$AA@  10002228     LIBCMT:nlsdata2.obj
 0001:0000122c       ??_C@_03HJBDCHOM@Feb?$AA@  1000222c     LIBCMT:nlsdata2.obj
 0001:00001230       ??_C@_03JIHJHPIE@Jan?$AA@  10002230     LIBCMT:nlsdata2.obj
 0001:00001234       ??_C@_08INBOOONO@Saturday?$AA@ 10002234     LIBCMT:nlsdata2.obj
 0001:00001240       ??_C@_06JECMNKMI@Friday?$AA@ 10002240     LIBCMT:nlsdata2.obj
 0001:00001248       ??_C@_08HACCIKIA@Thursday?$AA@ 10002248     LIBCMT:nlsdata2.obj
 0001:00001254       ??_C@_09DLIGFAKA@Wednesday?$AA@ 10002254     LIBCMT:nlsdata2.obj
 0001:00001260       ??_C@_07BAAGCFCM@Tuesday?$AA@ 10002260     LIBCMT:nlsdata2.obj
 0001:00001268       ??_C@_06JLEDEDGH@Monday?$AA@ 10002268     LIBCMT:nlsdata2.obj
 0001:00001270       ??_C@_06OOPIFAJ@Sunday?$AA@ 10002270     LIBCMT:nlsdata2.obj
 0001:00001278       ??_C@_03FEFJNEK@Sat?$AA@   10002278     LIBCMT:nlsdata2.obj
 0001:0000127c       ??_C@_03IDIOELNC@Fri?$AA@  1000227c     LIBCMT:nlsdata2.obj
 0001:00001280       ??_C@_03IOFIKPDN@Thu?$AA@  10002280     LIBCMT:nlsdata2.obj
 0001:00001284       ??_C@_03MHOMLAJA@Wed?$AA@  10002284     LIBCMT:nlsdata2.obj
 0001:00001288       ??_C@_03NAGEINEP@Tue?$AA@  10002288     LIBCMT:nlsdata2.obj
 0001:0000128c       ??_C@_03PDAGKDH@Mon?$AA@   1000228c     LIBCMT:nlsdata2.obj
 0001:00001290       ??_C@_03KOEHGMDN@Sun?$AA@  10002290     LIBCMT:nlsdata2.obj
 0001:00001294       ??_C@_0BK@CFCOFLF@?5Complete?5Object?5Locator?8?$AA@ 10002294     LIBCMT:undname.obj
 0001:000012b0       ??_C@_0BN@MECKDCOJ@?5Class?5Hierarchy?5Descriptor?8?$AA@ 100022b0     LIBCMT:undname.obj
 0001:000012d0       ??_C@_0BD@LGICGFMM@?5Base?5Class?5Array?8?$AA@ 100022d0     LIBCMT:undname.obj
 0001:000012e4       ??_C@_0BM@LDKODKLH@?5Base?5Class?5Descriptor?5at?5?$CI?$AA@ 100022e4     LIBCMT:undname.obj
 0001:00001300       ??_C@_0BC@DAFEJGAK@?5Type?5Descriptor?8?$AA@ 10002300     LIBCMT:undname.obj
 0001:00001314       ??_C@_0BM@PMGGMLDN@?$GAlocal?5static?5thread?5guard?8?$AA@ 10002314     LIBCMT:undname.obj
 0001:00001330       ??_C@_0CL@FGIJHLCE@?$GAmanaged?5vector?5copy?5constructor@ 10002330     LIBCMT:undname.obj
 0001:0000135c       ??_C@_0CJ@GJELGAMM@?$GAvector?5vbase?5copy?5constructor?5i@ 1000235c     LIBCMT:undname.obj
 0001:00001388       ??_C@_0CD@CGAJBKEJ@?$GAvector?5copy?5constructor?5iterato@ 10002388     LIBCMT:undname.obj
 0001:000013ac       ??_C@_0CB@PDBIFEP@?$GAdynamic?5atexit?5destructor?5for?5?8@ 100023ac     LIBCMT:undname.obj
 0001:000013d0       ??_C@_0BL@CLIPGLGB@?$GAdynamic?5initializer?5for?5?8?$AA@ 100023d0     LIBCMT:undname.obj
 0001:000013ec       ??_C@_0CM@FCBBDIGB@?$GAeh?5vector?5vbase?5copy?5constructo@ 100023ec     LIBCMT:undname.obj
 0001:00001418       ??_C@_0CG@HLDDJMAG@?$GAeh?5vector?5copy?5constructor?5iter@ 10002418     LIBCMT:undname.obj
 0001:00001440       ??_C@_0CF@IMGKMJNO@?$GAmanaged?5vector?5destructor?5itera@ 10002440     LIBCMT:undname.obj
 0001:00001468       ??_C@_0CG@CFDHKGGD@?$GAmanaged?5vector?5constructor?5iter@ 10002468     LIBCMT:undname.obj
 0001:00001490       ??_C@_0BN@CKNJLHMB@?$GAplacement?5delete?$FL?$FN?5closure?8?$AA@ 10002490     LIBCMT:undname.obj
 0001:000014b0       ??_C@_0BL@CNOONJFP@?$GAplacement?5delete?5closure?8?$AA@ 100024b0     LIBCMT:undname.obj
 0001:000014cc       ??_C@_0P@HJKNJFNN@?$GAomni?5callsig?8?$AA@ 100024cc     LIBCMT:undname.obj
 0001:000014dc       ??_C@_09LBNFPBCA@?5delete?$FL?$FN?$AA@ 100024dc     LIBCMT:undname.obj
 0001:000014e8       ??_C@_06FHBGPFGH@?5new?$FL?$FN?$AA@ 100024e8     LIBCMT:undname.obj
 0001:000014f0       ??_C@_0CE@IIHCMGGL@?$GAlocal?5vftable?5constructor?5closu@ 100024f0     LIBCMT:undname.obj
 0001:00001514       ??_C@_0BA@KKLDJDLB@?$GAlocal?5vftable?8?$AA@ 10002514     LIBCMT:undname.obj
 0001:00001524       ??_C@_05KHLCHHI@?$GARTTI?$AA@ 10002524     LIBCMT:undname.obj
 0001:0000152c       ??_C@_03KLGMFNMG@?$GAEH?$AA@ 1000252c     LIBCMT:undname.obj
 0001:00001530       ??_C@_0BA@KBCDOMBN@?$GAudt?5returning?8?$AA@ 10002530     LIBCMT:undname.obj
 0001:00001540       ??_C@_0BL@LLKPOHJI@?$GAcopy?5constructor?5closure?8?$AA@ 10002540     LIBCMT:undname.obj
 0001:0000155c       ??_C@_0CH@OOJPLCPH@?$GAeh?5vector?5vbase?5constructor?5ite@ 1000255c     LIBCMT:undname.obj
 0001:00001584       ??_C@_0CA@GCEOPDGL@?$GAeh?5vector?5destructor?5iterator?8?$AA@ 10002584     LIBCMT:undname.obj
 0001:000015a4       ??_C@_0CB@JONCMFFK@?$GAeh?5vector?5constructor?5iterator?8@ 100025a4     LIBCMT:undname.obj
 0001:000015c8       ??_C@_0BL@NILFHHPC@?$GAvirtual?5displacement?5map?8?$AA@ 100025c8     LIBCMT:undname.obj
 0001:000015e4       ??_C@_0CE@IKBNEHA@?$GAvector?5vbase?5constructor?5iterat@ 100025e4     LIBCMT:undname.obj
 0001:00001608       ??_C@_0BN@LFPFMEDL@?$GAvector?5destructor?5iterator?8?$AA@ 10002608     LIBCMT:undname.obj
 0001:00001628       ??_C@_0BO@PFGOCPJJ@?$GAvector?5constructor?5iterator?8?$AA@ 10002628     LIBCMT:undname.obj
 0001:00001648       ??_C@_0BN@IMDCHIKM@?$GAscalar?5deleting?5destructor?8?$AA@ 10002648     LIBCMT:undname.obj
 0001:00001668       ??_C@_0BO@OBMKPJIG@?$GAdefault?5constructor?5closure?8?$AA@ 10002668     LIBCMT:undname.obj
 0001:00001688       ??_C@_0BN@DEGPLNFK@?$GAvector?5deleting?5destructor?8?$AA@ 10002688     LIBCMT:undname.obj
 0001:000016a8       ??_C@_0BD@JDLKDPAB@?$GAvbase?5destructor?8?$AA@ 100026a8     LIBCMT:undname.obj
 0001:000016bc       ??_C@_08OBABFOLI@?$GAstring?8?$AA@ 100026bc     LIBCMT:undname.obj
 0001:000016c8       ??_C@_0BF@KDPPACIK@?$GAlocal?5static?5guard?8?$AA@ 100026c8     LIBCMT:undname.obj
 0001:000016e0       ??_C@_08LLFFHHDJ@?$GAtypeof?8?$AA@ 100026e0     LIBCMT:undname.obj
 0001:000016ec       ??_C@_07FEEIOKP@?$GAvcall?8?$AA@ 100026ec     LIBCMT:undname.obj
 0001:000016f4       ??_C@_09BLBHBJP@?$GAvbtable?8?$AA@ 100026f4     LIBCMT:undname.obj
 0001:00001700       ??_C@_09IFPLHPGF@?$GAvftable?8?$AA@ 10002700     LIBCMT:undname.obj
 0001:0000170c       ??_C@_02MHEGNOJ@?$FO?$DN?$AA@ 1000270c     LIBCMT:undname.obj
 0001:00001710       ??_C@_02DHLNPPGH@?$HM?$DN?$AA@ 10002710     LIBCMT:undname.obj
 0001:00001714       ??_C@_02FGJGFEAB@?$CG?$DN?$AA@ 10002714     LIBCMT:undname.obj
 0001:00001718       ??_C@_03CDNPDDLA@?$DM?$DM?$DN?$AA@ 10002718     LIBCMT:undname.obj
 0001:0000171c       ??_C@_03IKFCCPFF@?$DO?$DO?$DN?$AA@ 1000271c     LIBCMT:undname.obj
 0001:00001720       ??_C@_02FENAOKFI@?$CF?$DN?$AA@ 10002720     LIBCMT:undname.obj
 0001:00001724       ??_C@_02FJEHGPIO@?1?$DN?$AA@ 10002724     LIBCMT:undname.obj
 0001:00001728       ??_C@_02FKMDLLOA@?9?$DN?$AA@ 10002728     LIBCMT:undname.obj
 0001:0000172c       ??_C@_02FOEOMHFC@?$CL?$DN?$AA@ 1000272c     LIBCMT:undname.obj
 0001:00001730       ??_C@_02FPIMKNGF@?$CK?$DN?$AA@ 10002730     LIBCMT:undname.obj
 0001:00001734       ??_C@_02NONPIBCD@?$HM?$HM?$AA@ 10002734     LIBCMT:undname.obj
 0001:00001738       ??_C@_02PPKAJPJL@?$CG?$CG?$AA@ 10002738     LIBCMT:undname.obj
 0001:0000173c       ??_C@_01DNKMNLPK@?$HM?$AA@ 1000273c     LIBCMT:undname.obj
 0001:00001740       ??_C@_01JKBOJNNK@?$FO?$AA@ 10002740     LIBCMT:undname.obj
 0001:00001744       ??_C@_01PJKLJHI@?$HO?$AA@  10002744     LIBCMT:undname.obj
 0001:00001748       ??_C@_02HCKGKOFO@?$CI?$CJ?$AA@ 10002748     LIBCMT:undname.obj
 0001:0000174c       ??_C@_01IHBHIGKO@?0?$AA@   1000274c     LIBCMT:undname.obj
 0001:00001750       ??_C@_02EEKDKGMJ@?$DO?$DN?$AA@ 10002750     LIBCMT:undname.obj
 0001:00001754       ??_C@_01PPODPGHN@?$DO?$AA@ 10002754     LIBCMT:undname.obj
 0001:00001758       ??_C@_02EHCHHCKH@?$DM?$DN?$AA@ 10002758     LIBCMT:undname.obj
 0001:0000175c       ??_C@_01MNNFJEPP@?$DM?$AA@ 1000275c     LIBCMT:undname.obj
 0001:00001760       ??_C@_01FGNFDNOH@?$CF?$AA@ 10002760     LIBCMT:undname.obj
 0001:00001764       ??_C@_01KMDKNFGN@?1?$AA@   10002764     LIBCMT:undname.obj
 0001:00001768       ??_C@_03MNHNFDLC@?9?$DO?$CK?$AA@ 10002768     LIBCMT:undname.obj
 0001:0000176c       ??_C@_01HNPIGOCE@?$CG?$AA@ 1000276c     LIBCMT:undname.obj
 0001:00001770       ??_C@_01MIFGBAGJ@?$CL?$AA@ 10002770     LIBCMT:undname.obj
 0001:00001774       ??_C@_01JOAMLHOP@?9?$AA@   10002774     LIBCMT:undname.obj
 0001:00001778       ??_C@_02BAABKJLB@?9?9?$AA@ 10002778     LIBCMT:undname.obj
 0001:0000177c       ??_C@_02ECNGHCIF@?$CL?$CL?$AA@ 1000277c     LIBCMT:undname.obj
 0001:00001780       ??_C@_01NBENCBCI@?$CK?$AA@ 10002780     LIBCMT:undname.obj
 0001:00001784       ??_C@_02HBOOOICD@?9?$DO?$AA@ 10002784     LIBCMT:undname.obj
 0001:00001788       ??_C@_08LHJFAFGD@operator?$AA@ 10002788     LIBCMT:undname.obj
 0001:00001794       ??_C@_02GPECMEKF@?$FL?$FN?$AA@ 10002794     LIBCMT:undname.obj
 0001:00001798       ??_C@_02FDNJECIE@?$CB?$DN?$AA@ 10002798     LIBCMT:undname.obj
 0001:0000179c       ??_C@_02EGOFBIJA@?$DN?$DN?$AA@ 1000279c     LIBCMT:undname.obj
 0001:000017a0       ??_C@_01DCLJPIOD@?$CB?$AA@ 100027a0     LIBCMT:undname.obj
 0001:000017a4       ??_C@_02FODMEDOG@?$DM?$DM?$AA@ 100027a4     LIBCMT:undname.obj
 0001:000017a8       ??_C@_02GPIOPFAK@?$DO?$DO?$AA@ 100027a8     LIBCMT:undname.obj
 0001:000017ac       ??_C@_01NEMOKFLO@?$DN?$AA@ 100027ac     LIBCMT:undname.obj
 0001:000017b0       ??_C@_07FPCDHGMM@?5delete?$AA@ 100027b0     LIBCMT:undname.obj
 0001:000017b8       ??_C@_04NIHEBCM@?5new?$AA@ 100027b8     LIBCMT:undname.obj
 0001:000017bd       ??_C@_00CNPNBAHC@?$AA@     100027bd     LIBCMT:undname.obj
 0001:000017c0       ??_C@_0M@GFIIJFMG@__unaligned?$AA@ 100027c0     LIBCMT:undname.obj
 0001:000017cc       ??_C@_0L@PILCLIHE@__restrict?$AA@ 100027cc     LIBCMT:undname.obj
 0001:000017d8       ??_C@_07JOMMBBKO@__ptr64?$AA@ 100027d8     LIBCMT:undname.obj
 0001:000017e0       ??_C@_06GHPCKEAG@__eabi?$AA@ 100027e0     LIBCMT:undname.obj
 0001:000017e8       ??_C@_09HIJEGCPM@__clrcall?$AA@ 100027e8     LIBCMT:undname.obj
 0001:000017f4       ??_C@_0L@JMKHOMEK@__fastcall?$AA@ 100027f4     LIBCMT:undname.obj
 0001:00001800       ??_C@_0L@NPHFGOKO@__thiscall?$AA@ 10002800     LIBCMT:undname.obj
 0001:0000180c       ??_C@_09IFJBGAPI@__stdcall?$AA@ 1000280c     LIBCMT:undname.obj
 0001:00001818       ??_C@_08GHMPAG@__pascal?$AA@ 10002818     LIBCMT:undname.obj
 0001:00001824       ??_C@_07KOLFKCDI@__cdecl?$AA@ 10002824     LIBCMT:undname.obj
 0001:0000182c       ??_C@_08EHJDFFNH@__based?$CI?$AA@ 1000282c     LIBCMT:undname.obj
 0001:000019c8       ___newctype                100029c8     LIBCMT:ctype.obj
 0001:00001cc8       __wctype                   10002cc8     LIBCMT:ctype.obj
 0001:00001ed0       ___newclmap                10002ed0     LIBCMT:ctype.obj
 0001:00002050       ___newcumap                10003050     LIBCMT:ctype.obj
 0001:00002250       __load_config_used         10003250     LIBCMT:loadcfg.obj
 0001:00002298       ??_R4bad_alloc@std@@6B@    10003298     LIBCMT:new.obj
 0001:000022ac       ??_R3bad_alloc@std@@8      100032ac     LIBCMT:new.obj
 0001:000022bc       ??_R2bad_alloc@std@@8      100032bc     LIBCMT:new.obj
 0001:000022c8       ??_R1A@?0A@EA@bad_alloc@std@@8 100032c8     LIBCMT:new.obj
 0001:000022e4       ??_R1A@?0A@EA@exception@std@@8 100032e4     LIBCMT:new.obj
 0001:00002300       ??_R3exception@std@@8      10003300     LIBCMT:new.obj
 0001:00002310       ??_R2exception@std@@8      10003310     LIBCMT:new.obj
 0001:00002318       ??_R4exception@std@@6B@    10003318     LIBCMT:stdexcpt.obj
 0001:0000232c       ??_R4type_info@@6B@        1000332c     LIBCMT:typinfo.obj
 0001:00002340       ??_R3type_info@@8          10003340     LIBCMT:typinfo.obj
 0001:00002350       ??_R2type_info@@8          10003350     LIBCMT:typinfo.obj
 0001:00002358       ??_R1A@?0A@EA@type_info@@8 10003358     LIBCMT:typinfo.obj
 0001:00002380       ___safe_se_handler_table   10003380     <linker-defined>
 0001:0000238c       ___rtc_iaa                 1000338c     LIBCMT:_initsect_.obj
 0001:00002390       ___rtc_izz                 10003390     LIBCMT:_initsect_.obj
 0001:00002394       ___rtc_taa                 10003394     LIBCMT:_initsect_.obj
 0001:00002398       ___rtc_tzz                 10003398     LIBCMT:_initsect_.obj
 0001:000023a0       __alloca_probe             100033a0     chkstk.obj
 0001:000023a0       __chkstk                   100033a0 f   chkstk.obj
 0001:000023d0       _GetGlobalInfoW@4          100033d0 f   FileCase.obj
 0001:00002450       _SetStartupInfoW@4         10003450 f   FileCase.obj
 0001:000026c0       _OpenW@4                   100036c0 f   FileCase.obj
 0001:000026d0       _GetPluginInfoW@4          100036d0 f   FileCase.obj
 0001:00002710       ?GetLangString@PluginDialogBuilder@@MAEPB_WH@Z 10003710 f i filecvt.obj
 0001:00002730       ?DlgProc@@YGHPAXHH0@Z      10003730 f   filecvt.obj
 0001:00002780       ?InitDialogItem@?$DialogBuilderBase@UFarDialogItem@@@@MAEXPAUFarDialogItem@@PB_W@Z 10003780 f i filecvt.obj
 0001:00002780       ?SaveValue@?$DialogItemBinding@UFarDialogItem@@@@UAEXPAUFarDialogItem@@H@Z 10003780 f i filecvt.obj
 0001:00002790       ?TextWidth@?$DialogBuilderBase@UFarDialogItem@@@@MAEHABUFarDialogItem@@@Z 10003790 f i filecvt.obj
 0001:000027a0       ?DoShowDialog@?$DialogBuilderBase@UFarDialogItem@@@@MAEHXZ 100037a0 f i filecvt.obj
 0001:000027b0       ?AddUIntEditField@?$DialogBuilderBase@UFarDialogItem@@@@UAEPAUFarDialogItem@@PAIH@Z 100037b0 f i filecvt.obj
 0001:000027b0       ?CreateCheckBoxBinding@?$DialogBuilderBase@UFarDialogItem@@@@MAEPAU?$DialogItemBinding@UFarDialogItem@@@@PAHH@Z 100037b0 f i filecvt.obj
 0001:000027b0       ?AddIntEditField@?$DialogBuilderBase@UFarDialogItem@@@@UAEPAUFarDialogItem@@PAHH@Z 100037b0 f i filecvt.obj
 0001:000027c0       ?CreateRadioButtonBinding@?$DialogBuilderBase@UFarDialogItem@@@@MAEPAU?$DialogItemBinding@UFarDialogItem@@@@PAH@Z 100037c0 f i filecvt.obj
 0001:000027c0       ?GetLangString@?$DialogBuilderBase@UFarDialogItem@@@@MAEPB_WH@Z 100037c0 f i filecvt.obj
 0001:000027d0       ??1?$DialogBuilderBase@UFarDialogItem@@@@MAE@XZ 100037d0 f i filecvt.obj
 0001:00002820       ??_G?$DialogBuilderBase@UFarDialogItem@@@@MAEPAXI@Z 10003820 f i filecvt.obj
 0001:00002820       ??_E?$DialogBuilderBase@UFarDialogItem@@@@MAEPAXI@Z 10003820 f i filecvt.obj
 0001:00002840       ?ReallocDialogItems@?$DialogBuilderBase@UFarDialogItem@@@@IAEXXZ 10003840 f i filecvt.obj
 0001:00002910       ?UpdateSecondColumnPosition@?$DialogBuilderBase@UFarDialogItem@@@@IAEXXZ 10003910 f i filecvt.obj
 0001:00002970       ?SaveValues@?$DialogBuilderBase@UFarDialogItem@@@@IAEXXZ 10003970 f i filecvt.obj
 0001:000029c0       ?MaxTextWidth@?$DialogBuilderBase@UFarDialogItem@@@@IAEHXZ 100039c0 f i filecvt.obj
 0001:00002a80       ?SaveValue@PluginEditFieldBinding@@UAEXPAUFarDialogItem@@H@Z 10003a80 f i filecvt.obj
 0001:00002ab0       ?InitDialogItem@PluginDialogBuilder@@MAEXPAUFarDialogItem@@PB_W@Z 10003ab0 f i filecvt.obj
 0001:00002ad0       ?TextWidth@PluginDialogBuilder@@MAEHABUFarDialogItem@@@Z 10003ad0 f i filecvt.obj
 0001:00002af0       ?DoShowDialog@PluginDialogBuilder@@MAEHXZ 10003af0 f i filecvt.obj
 0001:00002b50       ?SaveValue@PluginCheckBoxBinding@@UAEXPAUFarDialogItem@@H@Z 10003b50 f i filecvt.obj
 0001:00002b90       ?SaveValue@PluginRadioButtonBinding@@UAEXPAUFarDialogItem@@H@Z 10003b90 f i filecvt.obj
 0001:00002bc0       ??0PluginIntEditFieldBinding@@QAE@ABUPluginStartupInfo@@PAPAXHPAHH@Z 10003bc0 f i filecvt.obj
 0001:00002c60       ?SaveValue@PluginIntEditFieldBinding@@UAEXPAUFarDialogItem@@H@Z 10003c60 f i filecvt.obj
 0001:00002c90       ??0PluginUIntEditFieldBinding@@QAE@ABUPluginStartupInfo@@PAPAXHPAIH@Z 10003c90 f i filecvt.obj
 0001:00002d30       ?SaveValue@PluginUIntEditFieldBinding@@UAEXPAUFarDialogItem@@H@Z 10003d30 f i filecvt.obj
 0001:00002d60       ?CreateCheckBoxBinding@PluginDialogBuilder@@MAEPAU?$DialogItemBinding@UFarDialogItem@@@@PAHH@Z 10003d60 f i filecvt.obj
 0001:00002db0       ?CreateRadioButtonBinding@PluginDialogBuilder@@MAEPAU?$DialogItemBinding@UFarDialogItem@@@@PAH@Z 10003db0 f i filecvt.obj
 0001:00002e00       ??_EPluginDialogBuilder@@UAEPAXI@Z 10003e00 f i filecvt.obj
 0001:00002e00       ??_GPluginDialogBuilder@@UAEPAXI@Z 10003e00 f i filecvt.obj
 0001:00002e40       ?AddCheckbox@?$DialogBuilderBase@UFarDialogItem@@@@QAEPAUFarDialogItem@@HPAHH_N@Z 10003e40 f i filecvt.obj
 0001:00002f70       ?AddRadioButtons@?$DialogBuilderBase@UFarDialogItem@@@@QAEXPAHHQBH_N@Z 10003f70 f i filecvt.obj
 0001:000030d0       ?AddButtonAfter@?$DialogBuilderBase@UFarDialogItem@@@@QAEPAUFarDialogItem@@PAU2@H@Z 100040d0 f i filecvt.obj
 0001:000031e0       ?EndColumns@?$DialogBuilderBase@UFarDialogItem@@@@QAEXXZ 100041e0 f i filecvt.obj
 0001:000032b0       ?AddSeparator@?$DialogBuilderBase@UFarDialogItem@@@@QAEXPB_W@Z 100042b0 f i filecvt.obj
 0001:00003320       ?AddButtons@?$DialogBuilderBase@UFarDialogItem@@@@QAEXHPBHHH@Z 10004320 f i filecvt.obj
 0001:00003480       ?UpdateBorderSize@?$DialogBuilderBase@UFarDialogItem@@@@IAEXXZ 10004480 f i filecvt.obj
 0001:00003530       ??_EPluginUIntEditFieldBinding@@UAEPAXI@Z 10004530 f i filecvt.obj
 0001:00003530       ??_E?$DialogItemBinding@UFarDialogItem@@@@UAEPAXI@Z 10004530 f i filecvt.obj
 0001:00003530       ??_GPluginRadioButtonBinding@@UAEPAXI@Z 10004530 f i filecvt.obj
 0001:00003530       ??_GPluginCheckBoxBinding@@UAEPAXI@Z 10004530 f i filecvt.obj
 0001:00003530       ??_EPluginCheckBoxBinding@@UAEPAXI@Z 10004530 f i filecvt.obj
 0001:00003530       ??_EPluginEditFieldBinding@@UAEPAXI@Z 10004530 f i filecvt.obj
 0001:00003530       ??_GPluginUIntEditFieldBinding@@UAEPAXI@Z 10004530 f i filecvt.obj
 0001:00003530       ??_EPluginRadioButtonBinding@@UAEPAXI@Z 10004530 f i filecvt.obj
 0001:00003530       ??_G?$DialogItemBinding@UFarDialogItem@@@@UAEPAXI@Z 10004530 f i filecvt.obj
 0001:00003530       ??_EPluginIntEditFieldBinding@@UAEPAXI@Z 10004530 f i filecvt.obj
 0001:00003530       ??_GPluginIntEditFieldBinding@@UAEPAXI@Z 10004530 f i filecvt.obj
 0001:00003530       ??_GPluginEditFieldBinding@@UAEPAXI@Z 10004530 f i filecvt.obj
 0001:00003550       ??0PluginDialogBuilder@@QAE@ABUPluginStartupInfo@@ABU_GUID@@1HPB_WP6GHPAXHH3@Z3_K@Z 10004550 f i filecvt.obj
 0001:00003660       ?AddIntEditField@PluginDialogBuilder@@UAEPAUFarDialogItem@@PAHH@Z 10004660 f i filecvt.obj
 0001:00003720       ?AddUIntEditField@PluginDialogBuilder@@UAEPAUFarDialogItem@@PAIH@Z 10004720 f i filecvt.obj
 0001:000037e0       ?AddEditField@PluginDialogBuilder@@QAEPAUFarDialogItem@@PA_WHHPB_W_N@Z 100047e0 f i filecvt.obj
 0001:000038e0       ?CaseConvertion@@YAXXZ     100048e0 f   filecvt.obj
 0001:000040e0       ?GetMsg@@YAPB_WH@Z         100050e0 f   FileMix.obj
 0001:00004100       ?IsCaseMixed@@YAHPB_W@Z    10005100 f   FileMix.obj
 0001:00004180       ?IsWordDiv@@YAHH@Z         10005180 f   FileMix.obj
 0001:000041b0       ?CaseWord@@YAXPA_WH@Z      100051b0 f   FileMix.obj
 0001:00004250       ?ProcessName@@YAXPB_WK@Z   10005250 f   ProcessName.obj
 0001:0000450a       ??3@YAXPAX@Z               1000550a f   LIBCMT:delete.obj
 0001:00004515       ??1bad_alloc@std@@UAE@XZ   10005515 f i LIBCMT:new.obj
 0001:00004520       ??_Gbad_alloc@std@@UAEPAXI@Z 10005520 f i LIBCMT:new.obj
 0001:00004520       ??_Ebad_alloc@std@@UAEPAXI@Z 10005520 f i LIBCMT:new.obj
 0001:00004547       ??0bad_alloc@std@@QAE@ABV01@@Z 10005547 f i LIBCMT:new.obj
 0001:00004564       ??2@YAPAXI@Z               10005564 f   LIBCMT:new.obj
 0001:000045f0       _memset                    100055f0 f   LIBCMT:memset.obj
 0001:0000466a       _free                      1000566a f   LIBCMT:free.obj
 0001:000046a4       _malloc                    100056a4 f   LIBCMT:malloc.obj
 0001:00004738       _wcsrchr                   10005738 f   LIBCMT:wcsrchr.obj
 0001:00004766       __CRT_INIT@12              10005766 f   LIBCMT:dllcrt0.obj
 0001:000049c0       __DllMainCRTStartup@12     100059c0 f   LIBCMT:dllcrt0.obj
 0001:000049e3       ??0exception@std@@QAE@ABQBDH@Z 100059e3 f   LIBCMT:stdexcpt.obj
 0001:00004a00       ?what@exception@std@@UBEPBDXZ 10005a00 f   LIBCMT:stdexcpt.obj
 0001:00004a0d       ?_Copy_str@exception@std@@AAEXPBD@Z 10005a0d f   LIBCMT:stdexcpt.obj
 0001:00004a4d       ?_Tidy@exception@std@@AAEXXZ 10005a4d f   LIBCMT:stdexcpt.obj
 0001:00004a6b       ??4exception@std@@QAEAAV01@ABV01@@Z 10005a6b f   LIBCMT:stdexcpt.obj
 0001:00004aa0       ??1exception@std@@UAE@XZ   10005aa0 f   LIBCMT:stdexcpt.obj
 0001:00004aab       ??_Gexception@std@@UAEPAXI@Z 10005aab f i LIBCMT:stdexcpt.obj
 0001:00004aab       ??_Eexception@std@@UAEPAXI@Z 10005aab f i LIBCMT:stdexcpt.obj
 0001:00004ad2       ??0exception@std@@QAE@ABV01@@Z 10005ad2 f   LIBCMT:stdexcpt.obj
 0001:00004af7       ??1type_info@@UAE@XZ       10005af7 f   LIBCMT:typinfo.obj
 0001:00004b07       ??_Etype_info@@UAEPAXI@Z   10005b07 f i LIBCMT:typinfo.obj
 0001:00004b07       ??_Gtype_info@@UAEPAXI@Z   10005b07 f i LIBCMT:typinfo.obj
 0001:00004bde       ___onexitinit              10005bde f   LIBCMT:onexit.obj
 0001:00004c0f       __onexit                   10005c0f f   LIBCMT:onexit.obj
 0001:00004c4b       _atexit                    10005c4b f   LIBCMT:onexit.obj
 0001:00004c62       __initp_heap_handler       10005c62 f   LIBCMT:handler.obj
 0001:00004c71       __callnewh                 10005c71 f   LIBCMT:handler.obj
 0001:00004c99       __CxxThrowException@8      10005c99 f   LIBCMT:throw.obj
 0001:00004ce5       __VEC_memzero              10005ce5 f   LIBCMT:p4_memset.obj
 0001:00004d9f       ___sse2_available_init     10005d9f f   LIBCMT:cpu_disp.obj
 0001:00004daf       __get_errno_from_oserr     10005daf f   LIBCMT:dosmap.obj
 0001:00004df1       __errno                    10005df1 f   LIBCMT:dosmap.obj
 0001:00004e04       __heap_init                10005e04 f   LIBCMT:heapinit.obj
 0001:00004e22       __heap_term                10005e22 f   LIBCMT:heapinit.obj
 0001:00004e36       ___crtCorExitProcess       10005e36 f   LIBCMT:crt0dat.obj
 0001:00004e61       ___crtExitProcess          10005e61 f   LIBCMT:crt0dat.obj
 0001:00004e79       __lockexit                 10005e79 f   LIBCMT:crt0dat.obj
 0001:00004e82       __unlockexit               10005e82 f   LIBCMT:crt0dat.obj
 0001:00004e8b       __init_pointers            10005e8b f   LIBCMT:crt0dat.obj
 0001:00004ebe       __initterm_e               10005ebe f   LIBCMT:crt0dat.obj
 0001:00004ee2       __cinit                    10005ee2 f   LIBCMT:crt0dat.obj
 0001:000050b9       __exit                     100060b9 f   LIBCMT:crt0dat.obj
 0001:000050cf       __cexit                    100060cf f   LIBCMT:crt0dat.obj
 0001:000050de       __amsg_exit                100060de f   LIBCMT:crt0dat.obj
 0001:000050fc       __GET_RTERRMSG             100060fc f   LIBCMT:crt0msg.obj
 0001:00005122       __NMSG_WRITE               10006122 f   LIBCMT:crt0msg.obj
 0001:000052d1       __FF_MSGBANNER             100062d1 f   LIBCMT:crt0msg.obj
 0001:0000530a       __encoded_null             1000630a f   LIBCMT:tidtable.obj
 0001:00005313       ___crtTlsAlloc@4           10006313 f   LIBCMT:tidtable.obj
 0001:0000531c       ___set_flsgetvalue         1000631c f   LIBCMT:tidtable.obj
 0001:00005350       __mtterm                   10006350 f   LIBCMT:tidtable.obj
 0001:0000538d       __initptd                  1000638d f   LIBCMT:tidtable.obj
 0001:00005441       __getptd_noexit            10006441 f   LIBCMT:tidtable.obj
 0001:000054ba       __getptd                   100064ba f   LIBCMT:tidtable.obj
 0001:000054d4       __freefls@4                100064d4 f   LIBCMT:tidtable.obj
 0001:00005603       __freeptd                  10006603 f   LIBCMT:tidtable.obj
 0001:00005671       __mtinit                   10006671 f   LIBCMT:tidtable.obj
 0001:000057ec       __malloc_crt               100067ec f   LIBCMT:crtheap.obj
 0001:00005831       __calloc_crt               10006831 f   LIBCMT:crtheap.obj
 0001:0000587d       __realloc_crt              1000687d f   LIBCMT:crtheap.obj
 0001:000058cb       __ioinit                   100068cb f   LIBCMT:ioinit.obj
 0001:00005b10       __ioterm                   10006b10 f   LIBCMT:ioinit.obj
 0001:00005b63       __setenvp                  10006b63 f   LIBCMT:stdenvp.obj
 0001:00005dd9       __setargv                  10006dd9 f   LIBCMT:stdargv.obj
 0001:00005e94       ___crtGetEnvironmentStringsA 10006e94 f   LIBCMT:a_env.obj
 0001:00005f2b       __RTC_Initialize           10006f2b f   LIBCMT:_initsect_.obj
 0001:00005f51       __RTC_Terminate            10006f51 f   LIBCMT:_initsect_.obj
 0001:00005f80       __SEH_prolog4              10006f80 f   LIBCMT:sehprolg4.obj
 0001:00005fc5       __SEH_epilog4              10006fc5 f   LIBCMT:sehprolg4.obj
 0001:00005fe0       __except_handler4          10006fe0 f   LIBCMT:chandler4.obj
 0001:0000616f       __XcptFilter               1000716f f   LIBCMT:winxfltr.obj
 0001:000062b9       ___CppXcptFilter           100072b9 f   LIBCMT:winxfltr.obj
 0001:000062d9       _DllMain@12                100072d9 f   LIBCMT:dllmain.obj
 0001:000062df       ___security_init_cookie    100072df f   LIBCMT:gs_support.obj
 0001:0000637a       _strcpy_s                  1000737a f   LIBCMT:strcpy_s.obj
 0001:000063e0       _strlen                    100073e0 f   LIBCMT:strlen.obj
 0001:0000646b       ?_Type_info_dtor@type_info@@CAXPAV1@@Z 1000746b f   LIBCMT:typname.obj
 0001:000064e0       _strcmp                    100074e0 f   LIBCMT:strcmp.obj
 0001:00006568       __msize                    10007568 f   LIBCMT:msize.obj
 0001:0000659b       __mtinitlocks              1000759b f   LIBCMT:mlock.obj
 0001:000065e5       __mtdeletelocks            100075e5 f   LIBCMT:mlock.obj
 0001:0000663c       __unlock                   1000763c f   LIBCMT:mlock.obj
 0001:00006653       __mtinitlocknum            10007653 f   LIBCMT:mlock.obj
 0001:00006715       __lock                     10007715 f   LIBCMT:mlock.obj
 0001:00006748       __initp_misc_invarg        10007748 f   LIBCMT:invarg.obj
 0001:00006757       __call_reportfault         10007757 f   LIBCMT:invarg.obj
 0001:00006880       __invoke_watson            10007880 f   LIBCMT:invarg.obj
 0001:000068a5       __invalid_parameter        100078a5 f   LIBCMT:invarg.obj
 0001:000068d2       __invalid_parameter_noinfo 100078d2 f   LIBCMT:invarg.obj
 0001:000068e2       ?terminate@@YAXXZ          100078e2 f   LIBCMT:hooks.obj
 0001:0000691b       __initp_eh_hooks           1000791b f   LIBCMT:hooks.obj
 0001:0000692c       __initp_misc_winsig        1000792c f   LIBCMT:winsig.obj
 0001:00006981       ___get_sigabrt             10007981 f   LIBCMT:winsig.obj
 0001:0000698e       _raise                     1000798e f   LIBCMT:winsig.obj
 0001:00006b31       __initp_misc_rand_s        10007b31 f   LIBCMT:rand_s.obj
 0001:00006b40       __initp_misc_purevirt      10007b40 f   LIBCMT:inithelp.obj
 0001:00006b4f       __initp_misc_cfltcvt_tab   10007b4f f   LIBCMT:cmiscdat.obj
 0001:00006b80       __ValidateImageBase        10007b80 f   LIBCMT:pesect.obj
 0001:00006bc0       __FindPESection            10007bc0 f   LIBCMT:pesect.obj
 0001:00006c10       __IsNonwritableInCurrentImage 10007c10 f   LIBCMT:pesect.obj
 0001:00006ccc       ___crtMessageBoxW          10007ccc f   LIBCMT:crtmboxw.obj
 0001:00006e38       _wcscat_s                  10007e38 f   LIBCMT:wcscat_s.obj
 0001:00006ead       _wcsncpy_s                 10007ead f   LIBCMT:wcsncpy_s.obj
 0001:00006f7a       _wcslen                    10007f7a f   LIBCMT:wcslen.obj
 0001:00006f95       _wcscpy_s                  10007f95 f   LIBCMT:wcscpy_s.obj
 0001:00006ff8       __set_error_mode           10007ff8 f   LIBCMT:errmode.obj
 0001:00007037       @__security_check_cookie@4 10008037 f   LIBCMT:secchk.obj
 0001:00007046       ___addlocaleref            10008046 f   LIBCMT:localref.obj
 0001:000070d5       ___removelocaleref         100080d5 f   LIBCMT:localref.obj
 0001:0000716e       ___freetlocinfo            1000816e f   LIBCMT:localref.obj
 0001:000072b9       __updatetlocinfoEx_nolock  100082b9 f   LIBCMT:localref.obj
 0001:00007306       ___updatetlocinfo          10008306 f   LIBCMT:localref.obj
 0001:000075a2       ___updatetmbcinfo          100085a2 f   LIBCMT:mbctype.obj
 0001:00007646       ??0_LocaleUpdate@@QAE@PAUlocaleinfo_struct@@@Z 10008646 f i LIBCMT:mbctype.obj
 0001:00007749       __setmbcp_nolock           10008749 f   LIBCMT:mbctype.obj
 0001:00007932       __setmbcp                  10008932 f   LIBCMT:mbctype.obj
 0001:00007acc       ___initmbctable            10008acc f   LIBCMT:mbctype.obj
 0001:00007aea       __calloc_impl              10008aea f   LIBCMT:calloc_impl.obj
 0001:00007b6c       _realloc                   10008b6c f   LIBCMT:realloc.obj
 0001:00007c6c       __ismbblead                10008c6c f   LIBCMT:ismbbyte.obj
 0001:00007c90       __local_unwind4            10008c90 f   LIBCMT:exsup4.obj
 0001:00007d66       __seh_longjmp_unwind4@4    10008d66 f   LIBCMT:exsup4.obj
 0001:00007d82       @_EH4_CallFilterFunc@8     10008d82 f   LIBCMT:exsup4.obj
 0001:00007d99       @_EH4_TransferToHandler@8  10008d99 f   LIBCMT:exsup4.obj
 0001:00007db2       @_EH4_GlobalUnwind2@8      10008db2 f   LIBCMT:exsup4.obj
 0001:00007dcb       @_EH4_LocalUnwind@16       10008dcb f   LIBCMT:exsup4.obj
 0001:00007de2       __crt_debugger_hook        10008de2 f   LIBCMT:dbghook.obj
 0001:00007dea       _abort                     10008dea f   LIBCMT:abort.obj
 0001:00007e20       _memcpy                    10008e20 f   LIBCMT:memcpy.obj
 0001:00008181       __freea                    10009181 f i LIBCMT:a_loc.obj
 0001:000081a1       __fptrap                   100091a1 f   LIBCMT:crt0fp.obj
 0001:000081aa       ___report_gsfailure        100091aa f   LIBCMT:gs_report.obj
 0001:000082b0       ___free_lc_time            100092b0 f   LIBCMT:inittime.obj
 0001:00008627       ___free_lconv_num          10009627 f   LIBCMT:initnum.obj
 0001:00008690       ___free_lconv_mon          10009690 f   LIBCMT:initmon.obj
 0001:00008975       ___crtLCMapStringA         10009975 f   LIBCMT:a_map.obj
 0001:00008aa2       ___crtGetStringTypeA       10009aa2 f   LIBCMT:a_str.obj
 0001:00008af0       __global_unwind2           10009af0 f   LIBCMT:exsup.obj
 0001:00008b55       __local_unwind2            10009b55 f   LIBCMT:exsup.obj
 0001:00008bd9       __abnormal_termination     10009bd9 f   LIBCMT:exsup.obj
 0001:00008bfc       __NLG_Notify1              10009bfc f   LIBCMT:exsup.obj
 0001:00008c05       __NLG_Notify               10009c05 f   LIBCMT:exsup.obj
 0001:00008c1c       __NLG_Dispatch             10009c1c     LIBCMT:exsup.obj
 0001:00008c1c       __NLG_Dispatch2            10009c1c     LIBCMT:exsup.obj
 0001:00008c24       __NLG_Call                 10009c24 f   LIBCMT:exsup.obj
 0001:00008c26       __NLG_Return2              10009c26     LIBCMT:exsup.obj
 0001:00008c30       __aulldvrm                 10009c30 f   LIBCMT:ulldvrm.obj
 0001:00008cc5       __VEC_memcpy               10009cc5 f   LIBCMT:p4_memcpy.obj
 0001:00008dd0       __alloca_probe_16          10009dd0 f   LIBCMT:alloca16.obj
 0001:00008de6       __alloca_probe_8           10009de6     LIBCMT:alloca16.obj
 0001:00008e00       __allmul                   10009e00 f   LIBCMT:llmul.obj
 0001:00008e40       _strcspn                   10009e40 f   LIBCMT:strcspn.obj
 0001:00008e90       _strpbrk                   10009e90 f   LIBCMT:strpbrk.obj
 0001:00008ed0       ___ascii_strnicmp          10009ed0 f   LIBCMT:_strnicm.obj
 0001:00008f32       _RtlUnwind@16              10009f32 f   kernel32:KERNEL32.dll
 0001:00008f50       __TI2?AVbad_alloc@std@@    10009f50     LIBCMT:new.obj
 0001:00008f60       __CTA2?AVbad_alloc@std@@   10009f60     LIBCMT:new.obj
 0001:00008f6c       __CT??_R0?AVbad_alloc@std@@@8??0bad_alloc@std@@QAE@ABV01@@Z12 10009f6c     LIBCMT:new.obj
 0001:00008f88       __CT??_R0?AVexception@std@@@8??0exception@std@@QAE@ABV01@@Z12 10009f88     LIBCMT:new.obj
 0001:00009174       __IMPORT_DESCRIPTOR_KERNEL32 1000a174     kernel32:KERNEL32.dll
 0001:00009188       __NULL_IMPORT_DESCRIPTOR   1000a188     kernel32:KERNEL32.dll
 0002:00000000       ??_R0?AVbad_alloc@std@@@8  1000b000     LIBCMT:new.obj
 0002:0000001c       ??_R0?AVexception@std@@@8  1000b01c     LIBCMT:new.obj
 0002:00000040       ??_R0?AVtype_info@@@8      1000b040     LIBCMT:typinfo.obj
 0002:000001c8       ___flsindex                1000b1c8     LIBCMT:tidtable.obj
 0002:000001cc       ___getvalueindex           1000b1cc     LIBCMT:tidtable.obj
 0002:000001d0       ___badioinfo               1000b1d0     LIBCMT:ioinit.obj
 0002:00000330       __cfltcvt_tab              1000b330     LIBCMT:cmiscdat.obj
 0002:00000358       ___security_cookie         1000b358     LIBCMT:gs_cookie.obj
 0002:0000035c       ___security_cookie_complement 1000b35c     LIBCMT:gs_cookie.obj
 0002:00000360       ___clocalestr              1000b360     LIBCMT:nlsdata2.obj
 0002:00000368       ___lc_time_c               1000b368     LIBCMT:nlsdata2.obj
 0002:000004d0       ___initiallocinfo          1000b4d0     LIBCMT:nlsdata2.obj
 0002:000005a8       ___ptlocinfo               1000b5a8     LIBCMT:nlsdata2.obj
 0002:000005b0       ___initialmbcinfo          1000b5b0     LIBCMT:mbctype.obj
 0002:000007d0       __mbctype                  1000b7d0     LIBCMT:mbctype.obj
 0002:000008d8       __mbcasemap                1000b8d8     LIBCMT:mbctype.obj
 0002:000009d8       ___ptmbcinfo               1000b9d8     LIBCMT:mbctype.obj
 0002:00000ad0       ___abort_behavior          1000bad0     LIBCMT:abort.obj
 0002:00000ae0       ___lconv_static_decimal    1000bae0     LIBCMT:lconv.obj
 0002:00000ae4       ___lconv_static_W_decimal  1000bae4     LIBCMT:lconv.obj
 0002:00000ae8       ___lconv_c                 1000bae8     LIBCMT:lconv.obj
 0002:00000b38       ___lconv                   1000bb38     LIBCMT:lconv.obj
 0002:00000b3c       ___globallocalestatus      1000bb3c     LIBCMT:glstatus.obj
 0002:00000b40       __pctype                   1000bb40     LIBCMT:ctype.obj
 0002:00000b44       __pwctype                  1000bb44     LIBCMT:ctype.obj
 0002:00000b50       __NLG_Destination          1000bb50     LIBCMT:exsup.obj
 0002:00000b70       ___mb_cur_max              1000bb70     LIBCMT:nlsdata1.obj
 0002:00000b74       ___decimal_point           1000bb74     LIBCMT:nlsdata1.obj
 0002:00000b78       ___decimal_point_length    1000bb78     LIBCMT:nlsdata1.obj
 0002:00000b80       ?Info@@3UPluginStartupInfo@@A 1000bb80     FileCase.obj
 0002:00000c08       ?FSF@@3UFarStandardFunctions@@A 1000bc08     FileCase.obj
 0002:00000cc8       ?Opt@@3UOptions@@A         1000bcc8     FileCase.obj
 0002:000010e4       ?ResetButtonID@@3HA        1000c0e4     filecvt.obj
 0002:000010e8       ?WordDivEditID@@3HA        1000c0e8     filecvt.obj
 0002:00001104       __aenvptr                  1000c104     LIBCMT:dllcrt0.obj
 0002:00001108       __wenvptr                  1000c108     LIBCMT:dllcrt0.obj
 0002:0000110c       ___error_mode              1000c10c     LIBCMT:dllcrt0.obj
 0002:00001110       ___app_type                1000c110     LIBCMT:dllcrt0.obj
 0002:00001114       ?_pnhHeap@@3P6AHI@ZA       1000c114     LIBCMT:handler.obj
 0002:00001118       __crtheap                  1000c118     LIBCMT:heapinit.obj
 0002:0000111c       __umaskval                 1000c11c     LIBCMT:crt0dat.obj
 0002:00001120       ___argc                    1000c120     LIBCMT:crt0dat.obj
 0002:00001124       ___argv                    1000c124     LIBCMT:crt0dat.obj
 0002:00001128       ___wargv                   1000c128     LIBCMT:crt0dat.obj
 0002:0000112c       __environ                  1000c12c     LIBCMT:crt0dat.obj
 0002:00001130       ___initenv                 1000c130     LIBCMT:crt0dat.obj
 0002:00001134       __wenviron                 1000c134     LIBCMT:crt0dat.obj
 0002:00001138       ___winitenv                1000c138     LIBCMT:crt0dat.obj
 0002:0000113c       __pgmptr                   1000c13c     LIBCMT:crt0dat.obj
 0002:00001140       __wpgmptr                  1000c140     LIBCMT:crt0dat.obj
 0002:00001144       __exitflag                 1000c144     LIBCMT:crt0dat.obj
 0002:00001148       __C_Termination_Done       1000c148     LIBCMT:crt0dat.obj
 0002:0000114c       __C_Exit_Done              1000c14c     LIBCMT:crt0dat.obj
 0002:00001778       __newmode                  1000c778     LIBCMT:_newmode.obj
 0002:0000177c       _gpFlsAlloc                1000c77c     LIBCMT:tidtable.obj
 0002:00001780       _gpFlsGetValue             1000c780     LIBCMT:tidtable.obj
 0002:00001784       _gpFlsSetValue             1000c784     LIBCMT:tidtable.obj
 0002:00001788       _gpFlsFree                 1000c788     LIBCMT:tidtable.obj
 0002:0000178c       __maxwait                  1000c78c     LIBCMT:crtheap.obj
 0002:000019f0       ___pInvalidArgHandler      1000c9f0     LIBCMT:invarg.obj
 0002:000019f4       ?__pInconsistency@@3P6AXXZA 1000c9f4     LIBCMT:hooks.obj
 0002:00001a10       ___pPurecall               1000ca10     LIBCMT:inithelp.obj
 0002:00001a2c       ___mbulinfo                1000ca2c     LIBCMT:mbctype.obj
 0002:00001a38       ___mbcodepage              1000ca38     LIBCMT:mbctype.obj
 0002:00001a3c       ___ismbcodepage            1000ca3c     LIBCMT:mbctype.obj
 0002:00001a40       ___mblcid                  1000ca40     LIBCMT:mbctype.obj
 0002:00001a58       ?pArgList@UnDecorator@@0PAVReplicator@@A 1000ca58     LIBCMT:undname.obj
 0002:00001a5c       ?pZNameList@UnDecorator@@0PAVReplicator@@A 1000ca5c     LIBCMT:undname.obj
 0002:00001a60       ?pTemplateArgList@UnDecorator@@0PAVReplicator@@A 1000ca60     LIBCMT:undname.obj
 0002:00001a64       ?gName@UnDecorator@@0PBDB  1000ca64     LIBCMT:undname.obj
 0002:00001a68       ?name@UnDecorator@@0PBDB   1000ca68     LIBCMT:undname.obj
 0002:00001a6c       ?outputString@UnDecorator@@0PADA 1000ca6c     LIBCMT:undname.obj
 0002:00001a70       ?maxStringLength@UnDecorator@@0HA 1000ca70     LIBCMT:undname.obj
 0002:00001a74       ?disableFlags@UnDecorator@@0KA 1000ca74     LIBCMT:undname.obj
 0002:00001a78       ?m_pGetParameter@UnDecorator@@0P6APADJ@ZA 1000ca78     LIBCMT:undname.obj
 0002:00001a7c       ?fExplicitTemplateParams@UnDecorator@@0_NA 1000ca7c     LIBCMT:undname.obj
 0002:00001a7d       ?fGetTemplateArgumentList@UnDecorator@@0_NA 1000ca7d     LIBCMT:undname.obj
 0002:00001da4       ___lconv_static_null       1000cda4     LIBCMT:lconv.obj
 0002:00001da8       ___lconv_static_W_null     1000cda8     LIBCMT:lconv.obj
 0002:00001dac       ___locale_changed          1000cdac     LIBCMT:setlocal.obj
 0002:00001db0       __debugger_hook_dummy      1000cdb0     <common>
 0002:00001db4       __pDestructExceptionObject 1000cdb4     <common>
 0002:00001db8       __nhandle                  1000cdb8     <common>
 0002:00001dc0       ___pioinfo                 1000cdc0     <common>
 0002:00001ec0       ___env_initialized         1000cec0     <common>
 0002:00001ec4       ___onexitend               1000cec4     <common>
 0002:00001ec8       ___onexitbegin             1000cec8     <common>
 0002:00001ecc       ___mbctype_initialized     1000cecc     <common>
 0002:00001ed0       __FPinit                   1000ced0     <common>
 0002:00001ed4       ___dyn_tls_init_callback   1000ced4     <common>
 0002:00001ed8       ___sse2_available          1000ced8     <common>
 0002:00001edc       __acmdln                   1000cedc     <common>

 entry point at        0001:000049c0

 Static symbols

 0001:000048ca       ___DllMainCRTStartup       100058ca f   LIBCMT:dllcrt0.obj
 0001:00004b28       __onexit_nolock            10005b28 f   LIBCMT:onexit.obj
 0001:00004f79       _doexit                    10005f79 f   LIBCMT:crt0dat.obj
 0001:00005c3f       _parse_cmdline             10006c3f f   LIBCMT:stdargv.obj
 0001:0000694a       _siglookup                 1000794a f   LIBCMT:winsig.obj
 0001:0000737f       ?CPtoLCID@@YAHH@Z          1000837f f   LIBCMT:mbctype.obj
 0001:000073ae       ?setSBCS@@YAXPAUthreadmbcinfostruct@@@Z 100083ae f   LIBCMT:mbctype.obj
 0001:00007412       ?setSBUpLow@@YAXPAUthreadmbcinfostruct@@@Z 10008412 f   LIBCMT:mbctype.obj
 0001:000076cd       ?getSystemCP@@YAHH@Z       100086cd f   LIBCMT:mbctype.obj
 0001:00007c19       ?x_ismbbtype_l@@YAHPAUlocaleinfo_struct@@IHH@Z 10008c19 f   LIBCMT:ismbbyte.obj
 0001:00007d20       __unwind_handler4          10008d20 f   LIBCMT:exsup4.obj
 0001:0000878e       ?__crtLCMapStringA_stat@@YAHPAUlocaleinfo_struct@@KKPBDHPADHHH@Z 1000978e f   LIBCMT:a_map.obj
 0001:000089bb       ?__crtGetStringTypeA_stat@@YAHPAUlocaleinfo_struct@@KPBDHPAGHHH@Z 100099bb f   LIBCMT:a_str.obj
 0001:00008b10       __unwind_handler           10009b10 f   LIBCMT:exsup.obj
 0001:00008f38       ??__Fnomem@?5???2@YAPAXI@Z@YAXXZ 10009f38 f   LIBCMT:new.obj
